:020000040000FA
:04000000FAEF01F022
:08000800E8CF05F0D8CF06F0A7
:10001000E0CF07F00001E9CF0DF0EACF08F0E1CF23
:1000200009F0E2CF0AF0D9CF0BF0DACF0CF0F3CF22
:1000300014F0F4CF15F0FACF16F000C00FF001C0A5
:1000400010F002C011F003C012F004C013F09DAA1A
:100050002DEF00F09EBA9EEF00F00FC000F010C030
:1000600001F011C002F012C003F013C004F00DC083
:10007000E9FF08C0EAFF09C0E1FF0AC0E2FF0BC0C8
:10008000D9FF0CC0DAFF14C0F3FF15C0F4FF16C08F
:10009000FAFF05C0E8FF07C0E0FF06C0D8FF100068
:1000A000F2CF0EF0F29EF76ABA0FF66E000EF7224C
:1000B0000900F5500EBEF28E12000A0D496E6974E9
:1000C00069616C697A696E6720506F727420420AA8
:1000D0000D00F2CF0EF0F29EF76AEC0FF66E000EF6
:1000E000F7220900F5500EBEF28E1200436F6E66C5
:1000F00069677572696E672052462D3234470A0D62
:100100000000F2CF0EF0F29EF76A1C0FF66E010EA1
:10011000F7220900F5500EBEF28E12004F4B210A55
:100120000D0A0D009EAAFED7ABCF18F0AECF01F09E
:1001300018A202D0AB98AB880000000CF3DF01C01E
:1001400023F02350120A03E0770A26E02DD0EADFDD
:100150000150340802E0000E01D0010E256EE2DFEE
:100160000150560802E0000E01D0010E2514276E42
:10017000D9DF0150780802E0000E01D0010E2714EB
:10018000296ED0DF0150900802E0000E01D0010E70
:100190002914D8A4FF0008D0C5DF01C019F0C2DFC0
:1001A00001C01AF01B8000D09E9A2DEF00F0EA6A81
:1001B0001C0EE96EEF500FE0030E016E006A002E78
:1001C000FED7012EFBD73C0E006E002EFED700009E
:1001D0000000EF2EF1D7000C070E206E1F6A1F5093
:1001E00007081DE3939A8A9A20502006216E1EC0AC
:1001F00000F02150016E04E0D8900032012EFCD7AF
:1002000000A003D093988A8802D093988A9800001F
:100210000000939A8A8A000000001F2AE0D7000C91
:1002200093968A96939E8A9E939A8A9A93988A988E
:10023000030E1C6EBCDF939E8A8E080E006E002E8D
:10024000FED7100E1E6EC8DF100E1E6EC5DF1E6AB2
:10025000C3DF1E6AC1DF1E6ABFDF420E1E6EBCDF37
:10026000420E1E6EB9DF1E6AB7DF1E6AB5DF1E6A58
:10027000B3DF420E1E6EB0DF420E1E6EADDF430EC8
:100280001E6EAADF6F0E1E6EA7DF810E1E6EA4DF2C
:10029000938893968A96939E8A9E939A8A9A69EFF8
:1002A00002F093968A96939E8A8E080E006E002E18
:1002B000FED793988A88939A8A8A00000000939ABE
:1002C0008A9A00000000939E8A9E9388939A8A9A45
:1002D00093968A86000C206A070E216E1F6A1F50B3
:1002E00007082BE3939A8A9A00000000939A8A8A5F
:1002F00000000000938881A80FD021502106226EB3
:10030000010E006E2250016E04E0D8900036012EDE
:10031000FCD7005020120FD021502106226E010E72
:10032000006E2250016E04E0D8900036012EFCD7FA
:100330000050FF0A20161F2AD2D720C001F0B0EFCC
:1003400001F01C6A1C50010813E3036A1C50190FCA
:10035000016E000E032201C01DF003C01EF0BBD7CA
:100360001EC0EAFF1DC0E9FF01C0EFFF1C2AEAD74B
:10037000939A8A9A93968A867DEF02F093968A964C
:10038000939E8A8E080E006E002EFED793988A9850
:10039000939A8A8A00000000939A8A9A00000000CB
:1003A000939E8A9E939A8A9A8CEF02F093968A86FD
:1003B000080E006E002EFED7420E1E6E0DDF420E9E
:1003C0001E6E0ADF1C6A1C5001080EE3036A1C50F3
:1003D000190FE96E000E0320EA6EEFCF1DF01DC06D
:1003E0001EF0FADE1C2AEFD793968A96939A8A9A81
:1003F00090EF02F0F86AD09E0D8EEA6AE96AB8863C
:100400002A0EAF6E000EB06E260EAC6E900EAB6E66
:10041000C150C00B0F09C16E070EB46E186A1B9055
:10042000C150C00B0F09C16EC290880ED56ECD6A47
:10043000000ECA6E7F0ECB6EB150480BB16EB70E78
:10044000B1169484BD6ABD6AB1169482BA6ABA6A5A
:100450009D8AC00EF212640E1C6EA9DE1C6A1C502E
:100460001FDE1C2A006E00509EA8FED7AD6E150E32
:100470001C5CF5E1030E1D6E2E0E9EA8FED7AD6E20
:100480001D2EFAD70A0E9EA8FED7AD6E0D0E9EA8A1
:10049000FED7AD6EF18EF2961C6A1C501ADE1C2A35
:1004A000006E00509EA8FED7AD6E120E1C5CF5E1EA
:1004B000030E1D6E2E0E9EA8FED7AD6E1D2EFAD712
:1004C0000A0E9EA8FED7AD6E0D0E9EA8FED7AD6E8D
:1004D000A7D6E7DE7F0E196E1A6E1C6A1C5011DE5D
:1004E0001C2A006E00509EA8FED7AD6E070E1C5C45
:1004F000F5E1938C81AC0DD024D7650E9EA8FED774
:10050000AD6E19509EA8FED7AD6E1A509EA8FED7AC
:10051000AD6E1BA00DD032D7010E1C6E48DE46D743
:10052000010E1C6E44DEBDDE010E1C6E40DE1B9013
:04053000E0D703000D
:00000001FF
